:020000040001F9
:1090000078270020F99201000193010003930100E9
:10901000059301000793010009930100000000007F
:109020000000000000000000000000000B930100A1
:109030000D930100000000000F9301001193010047
:10904000F1950100139301001393010013930100A4
:109050001393010000000000299401001393010004
:109060001393010013930100139301001393010064
:109070001393010013930100139301001393010054
:10908000139301004996010013930100139301000B
:109090006D96010013930100719601001393010076
:1090A0001393010013930100000000000000000072
:1090B0001393010013930100000000000000000062
:1090C00000000000000000000000000000000000A0
:1090D0000000000000000000000000000000000090
:1090E0000000000000000000000000000000000080
:1090F0000000000000000000000000000000000070
:10910000000000000000000000000000000000005F
:10911000000000000000000000000000000000004F
:10912000000000000000000000000000000000003F
:10913000000000000000000000000000000000002F
:10914000000000000000000000000000000000001F
:10915000000000000000000000000000000000000F
:1091600000000000000000000000000000000000FF
:1091700000000000000000000000000000000000EF
:1091800000000000000000000000000000000000DF
:1091900000000000000000000000000000000000CF
:1091A00000000000000000000000000000000000BF
:1091B00000000000000000000000000000000000AF
:1091C000000000000000000000000000000000009F
:1091D000000000000000000000000000000000008F
:1091E000000000000000000000000000000000007F
:1091F000000000000000000000000000000000006F
:10920000DFF80CD000F0FEF8004800478DA90100FF
:109210007827002030B4044654E8000F0D4644E897
:109220000053002BF8D1156030BC704730B40446B1
:1092300054E8000F40EA010544E80053002BF7D141
:10924000156030BC704730B4044654E8000F00EAA3
:10925000010544E80053002BF7D1156030BC70477E
:1092600030B4044654E8000F80EA010544E8005396
:10927000002BF7D1156030BC704730B4044654E879
:10928000000F00EB010544E80053002BF7D11560F7
:1092900030BC704730B4044654E8000FA0EB010521
:1092A00044E80053002BF7D1156030BC704770B410
:1092B00004464FF0000054E8006F0D68AE4207BF4F
:1092C00044E80023012044E800630E60002B1CBF2B
:1092D0000020F0E770BC704730B4044654E8000F3B
:1092E00088422CBF451A054644E80053002BF5D1AF
:1092F000156030BC704700000648804706480047AC
:10930000FEE7FEE7FEE7FEE7FEE7FEE7FEE7FEE735
:10931000FEE7FEE775960100019201002DE9F05F7E
:109320000546002092469B468846064681464024D4
:109330001BE0284641464746224600F053F8534674
:109340005A46C01A914110D311461846224600F0E1
:1093500016F82D1A67EB01084F462246012000211E
:1093600000F00DF817EB00094E41201EA4F1010496
:10937000DFDC484631462A464346BDE8F09F202AB6
:1093800004DB203A00FA02F1002070479140C2F15C
:10939000200320FA03F319439040704740EA010389
:1093A0009B0703D009E008C9121F08C0042AFAD29B
:1093B00003E011F8013B00F8013B521EF9D270475F
:1093C000D2B201E000F8012B491EFBD27047002207
:1093D000F6E710B513460A4604461946FFF7F0FFB4
:1093E000204610BD202A04DB203A21FA02F0002199
:1093F000704721FA02F3D040C2F1200291400843A5
:1094000019467047064C074D06E0E06840F001033E
:1094100094E8070098471034AC42F6D3FFF7F4FE07
:10942000B4BC0100D4BC01002DE9F04700268AB08D
:10943000DFF85091B0464FF4807501243746069608
:10944000284601F0D9FD38B1D9F80403204203D0F1
:10945000284601F0C7FD26432D1D64007F1CADB2D8
:10946000082FEDD34FF4BE74204601F0C5FD48B17E
:10947000204601F0B7FD46F0004606AA0121002073
:1094800001F09CFD404D16F0FF0F15D00127002480
:1094900037420DD009EB8401D1F81005D1F8101531
:1094A000C0F3042055F82420C1F3014102B19047D4
:1094B0007F00641C082CEBD3002E5FDA4FF0FF30E6
:1094C000CDF8108054E0281910F8507F90F9000072
:1094D00027F0C008401C3BD007A9404601F0C9FB5B
:1094E00010B34FEA9719404600F08EFF55F82070F0
:1094F0001FB1B9F1030F03D006E0B9F1030F27D173
:1095000004A9404601F0BDFB4FF0A04101EB8800EB
:10951000D0F8000706A9C0F3014A404601F0A9FBB4
:1095200018B1BAF1020F03D012E0BAF1030F0FD154
:10953000B9F1030F08D1BAF1020F1DD00221404644
:1095400001F020FD761CF6B217B149464046B847F7
:10955000641C042CB7D3002E10D06A4601210020D1
:1095600001F02CFD06990098884207D006900498D7
:10957000002634460790A6E70321E0E70AB0BDE8DD
:10958000F087000000600040D41D002000F01F02A2
:10959000012191404009800000F1E020C0F88012D4
:1095A000704700F01F02012191404009800000F146
:1095B000E020C0F80011704700F01F020121914027
:1095C0004009800000F1E020C0F800127047490710
:1095D000090E002806DA00F00F0000F1E02080F804
:1095E000141D704700F1E02080F80014704700005F
:1095F00070B54FF48076304601F05CFC114CB50537
:1096000060B1304601F05DFC0120C5F808036079C7
:1096100020B9012060712168002088474FF48276CC
:10962000304601F047FC00280AD0304601F049FCE2
:109630000220C5F808032168BDE8704001200847F2
:1096400070BD0000481C002007480021C0F84011F0
:10965000C0F84411C0F84811C0F84C11C0F800110E
:10966000C0F8041102F0B8B90010014002F002B9CC
:1096700001F0D0BDF0B5A848A74B012600781B1D0E
:109680001A1D4FF0805106280BD11C78240708D1F1
:109690001478C4F30314032C06D0042C04D0052C36
:1096A00002D0062807D011E0B1F824439B4DC4F343
:1096B00004242C6002E01C78240707D11478C4F33A
:1096C0000314032C02D1974D954C6C67D1F830519F
:1096D000D1F84442944FC4F342343C6006280CD184
:1096E0001C78240709D11478C4F30314032C04D183
:1096F0008E4C276827F0807727604FF08047002442
:10970000C7F80C41C7F81041874F3F1F3C6006283F
:1097100007D11F783F0704D11778C7F30317032F2A
:1097200002D0062808D01FE0DFF8FCC103270CF1A7
:10973000640CCCF8007007E01F783F0714D117784D
:10974000C7F30317032F0FD1DFF8E4C10527CCF8C7
:109750000070774F78373E60754F08373C600CF1EA
:10976000040C3F27CCF80070724F3F68DFF8C8C187
:10977000CCF800706F4F3F1D3F680CF1040CCCF823
:1097800000706C4F08373F680CF1040CCCF8007087
:10979000684F0C373F680CF1040CCCF80070654F33
:1097A00010373F680CF1040CCCF80070614F14378F
:1097B0003F680CF1040CCCF800705E4F18373F681E
:1097C000DFF874C10CF1200CCCF80070594F1C3735
:1097D0003F680CF1040CCCF80070564F20373F68FE
:1097E0000CF1040CCCF80070524F24373F680CF198
:1097F000040CCCF800704F4F28373F680CF1040C74
:10980000CCF800704B4F2C373F680CF1040CCCF8AF
:109810000070484F30373F68DFF81CC10CF1400C36
:10982000CCF80070434F34373F680CF1040CCCF88F
:109830000070404F38373F680CF1040CCCF80070D2
:109840003C4F3C373F680CF1040CCCF80070394FAA
:1098500040373F680CF1040CCCF80070DFF8DCC036
:10986000FB27CCF80070062813D11F783F0710D1D2
:109870001778C7F30317032F03D0042F01D0052F48
:1098800007D1D1F85872DFF8B8C007F04F07CCF80D
:1098900000702C480268D20702D06FF0010202600B
:1098A000062D08D1D1F83401062804D126480168D4
:1098B00041F4806101604FF01021D1F800020028CE
:1098C00003DBD1F80402002822DA204A166020487F
:1098D0000368002BFCD01523C1F800320568002D69
:1098E000FCD0C1F8043201680029FCD01460016882
:1098F0000029FCD0BFF34F8F0C48F0380168154A9F
:1099000001F4E06111430160BFF34F8F00BFFDE739
:10991000124911480860F0BDE00F00F040350140E9
:109920000DF0ADBA00C007403C050040FCED00E082
:10993000105600400404001020C5004018F50040F7
:10994000E40E0040000400403C17004004E50140E4
:1099500000E401400400FA050090D003901C0020B0
:1099600002E008C8121F08C1002AFAD170477047E8
:10997000002001E001C1121F002AFBD17047000046
:109980000121202803DA81400548014003E04028F6
:1099900002DA2038814009B1012070470020704769
:1099A000FC06FFBD082806D228B1012803D00428F0
:1099B00001D00120704700207047000010B592B020
:1099C00005243C216846FFF702FD5920ADF83C0014
:1099D0001820ADF84000124811900FA8114A0990C4
:1099E0008DF8034002CA684600F076F908B100F02D
:1099F00085F80C480A4A10382C3A807840B109485A
:109A000000210D3872DF07E000F078F812B010BDC9
:109A10000449A1F10D0072DF0028F5D1F6E700003E
:109A20001C1D0020281C0020022000F0D1BA0000DC
:109A300070B50024064D06E06868012110F8340076
:109A400001F082FC641C28788442F5D3002070BDAC
:109A5000501C0020F8B515460C460646052A01D2D2
:109A60000720F8BD01F06CFD18B901F031FD0028A8
:109A7000F7D1124900224E600C708D60C1E90422BA
:109A8000C1E906220E4D0DE006EBC40029680091E5
:109A900081788DF8011000780A4A694601F0A6FC29
:109AA0000028DED1641EE4B2EED2BDE8F8400448DE
:109AB0000021054A001D00F02DB80000501C0020B8
:109AC000DCBB0100BDA70100E5A6010072B6094894
:109AD0000068C00700D000BEBFF34F8F0548E438D0
:109AE0000168054A01F4E06111430160BFF34F8F43
:109AF00000BFFDE7F0ED00E00400FA050EB500211F
:109B00000091CDE901106A4644F20100FFF7DEFF43
:109B10000EBD0000074B9B7823B12AB120B100682D
:109B2000037C1BB1082070470720704741744261D5
:109B300000207047501E002070B501F055FD104800
:109B400000240B21047044700E4D817014206C6051
:109B50002C706C70FFF71AFD07211420FFF737FDFA
:109B60001420FFF71EFD0848046007211120FFF7AD
:109B70002EFD0548001F0068A860002070BD000091
:109B8000501E0020701C0020081501402DE9FC47E4
:109B9000DFF8789099F8023073B368B3052902D2E0
:109BA0000720BDE8FC87436933B3437C012B25D0F4
:109BB000002704460025884616468DF80050684662
:109BC00000F038F801A801F059FFC8B10121017077
:109BD0000F4944600968C0E90218C0E904769DF89D
:109BE000040089F801009DF8000000F047F81420F7
:109BF000FFF7E2FC2846D4E70820D2E70F46D8E773
:109C000004259DF8000000F039F8F3E7501E00200D
:109C1000041501400649897839B130B1416921B153
:109C200000210174022101F0B3BE0820704700003A
:109C3000501E002030B5EFF3108172B60D4A9468C3
:109C4000012324B10370002900D162B630BD9360B6
:109C50004FF0E023D3F88051074C25401560C3F83E
:109C60008041D3F8844154605A17C3F884210022FC
:109C70000270E8E75C1F0020FC06FFBD0B498A6804
:109C8000002A11D000280FD1EFF3108072B60B68B4
:109C90004FF0E022C2F800314B68C2F804310022D4
:109CA0008A60002800D162B6704700005C1F002067
:109CB00010B5084C6068FFF7ADFF08B1FFF71EFF55
:109CC0002068FFF7A7FF002803D0BDE81040FFF78A
:109CD00015BF10BD7CBB01002DE9FC47002517888E
:109CE0000646158090F82D001446894630B13A4654
:109CF0002146484600F0B1F8051E09D1B0784FF072
:109D00000C0A18B32088C846001DB84202D9504634
:109D1000BDE8FC87684679DF0028F9D12088032157
:109D200008F8001020881921401C80B2208008F813
:109D300000102088401C80B2208000EB0801BDF894
:109D4000000001F083FE218808442080F078022280
:109D5000C8B1218896F9033001F1030C4846BC458F
:109D6000D5D8425421884FF0010C491C89B221807A
:109D700000F801C02188491C89B2218009F801300E
:109D80002088401C20807068B8B1218890F900308C
:109D900001F1030C4846BC45B9D8425421880A2237
:109DA000491C89B2218042542188491C89B22180F2
:109DB00009F801302088401C2080308950B1CDE95D
:109DC00000474B460622022106F1080001F06EFE14
:109DD000051E9DD1308A50B1CDE900474B46072280
:109DE000032106F1100001F061FE051E90D1308BB9
:109DF00050B1CDE900474B461522142106F1180059
:109E000001F054FE051E83D1306A30B13B46224634
:109E1000494600F021FC051EDBD1706A30B13B469B
:109E20002246494600F088FE051ED2D196F82C0045
:109E300038B13B4622464946304601F06BFC051ED0
:109E4000C7D1307838B13B4622464946304600F00B
:109E5000A5FE051EBDD128465AE77CB505460888F3
:109E60000C460930904201D90C207CBD68466DDF5C
:109E70000028FAD121880820685420881B21401C22
:109E800080B2208029542088401C80B22080284441
:109E9000DDF801100160BDF8051081802088801D6B
:109EA00080B220809DF80010490800D0012129547B
:109EB0002088401C208000207CBD000038B501882F
:109EC000224C3B2939D00CDC102914D0112918D090
:109ED000212922D0262929D1007A012826D133DF51
:109EE00015E050292DD0522921D056291ED1808825
:109EF000132176DF0BE08188A180154800F062FF16
:109F000005E04FF6FF70A080FFF7D2FE33DF002898
:109F10000CD0BDE83840FFF7F1BD002100918088EA
:109F200069468FDF002801D0FFF7E8FD38BD032325
:109F300000221146A088B1DFE9E78088132176DF8F
:109F4000E5E7BDE8384001F005BB0000181C002023
:109F5000E41C0020007800F0010070470649095C0D
:109F60004FF0A040D0F81005C84010F0010000D01C
:109F7000012080F00100704798BB01002DE9FC41F1
:109F80000646C0074FF000050ED0104F00240122F6
:109F9000385D009500231146019500F0CFFF641C49
:109FA000042CF4D300F046F8B0070DD5074E00247A
:109FB000361D0022305D032300951146019500F007
:109FC000BDFF641C042CF4D3BDE8FC8194BB0100EC
:109FD00007490B5C4FF0A041D1F8042501209840BF
:109FE00020EA0203C1F808351040C1F80C0570479B
:109FF00094BB01000249085C012100F0D4BF0000BD
:10A0000094BB01000249085C002100F0CCBF0000B5
:10A0100094BB01000649095C4FF0A040D0F804054C
:10A02000C84010F0010000D0012080F0010070470E
:10A0300094BB010010B500242046FFF7DBFF641C31
:10A04000042CF9D310BD10B500242046FFF7DAFF29
:10A05000641C042CF9D310BD10B50246064B4FF01A
:10A06000FF3000215C5C944201D1084610BD491CC0
:10A070000429F7D310BD000098BB01002DE9F0477B
:10A080000D468146FFF7E8FF0446042836D2DFF884
:10A0900074801B481C4EA8F10C0725B3012D0ED06F
:10A0A000022D2BD104EB440030444578002D25D0FF
:10A0B000B968002922D02846BDE8F047084704EBDC
:10A0C0004401755C0E44717849B10E4A4FF4004169
:10A0D000093A8068FFF75AFD08B987F80390B1780C
:10A0E00008F80410E2E78068FFF794FD04EB4401F0
:10A0F000314418F804008D78A842D7D0BDE8F08725
:10A100009CBB0100441C0020941D002070B500235E
:10A11000042810D20D4D00EB4004012A02D1012980
:10A120000CD00022094E00EB4000304461B10129FF
:10A1300006D0022906D00723184670BD0E30C2B2E1
:10A140002A55F9E74270F7E78270F5E7941D002081
:10A1500070B506461E480024C0E90161B00720D54D
:10A160000025012211462846FFF7D0FF6D1C04464A
:10A17000042D02D2002CF4D013E094B940F26662B0
:10A1800004211448FFF766FC04000AD1FFF750FCD5
:10A19000040006D10F48104A0021001FFFF7BAFC47
:10A1A0000446F00712D00120FFF7E8FE74B9094811
:10A1B0000A4A00210C38FFF7ADFC040006D105481F
:10A1C000074A01210838FFF7A5FC0446204670BD68
:10A1D000381C0020A8BB01009DA3010071A801004C
:10A1E000299A01002DE9F05F6A4C05460026607847
:10A1F000B34618B184F801B000F022FB664F4FF46B
:10A200007A694FF4C87A4FF00108182D62D2DFE85E
:10A2100005F0AC0C0C31404D62676B746B74BE7D05
:10A220007D7D7D7DACAFB2B5BEBE0020FFF7F2FEF6
:10A2300000284FF0000008D0FFF7DCFE022D02D10D
:10A240004FF4E16008E0484606E0FFF7DBFE022D30
:10A2500001D1C82000E05046410CC0034FF4FA720F
:10A26000801841F10001257052000023FFF756F8D5
:10A2700001462AE00020FFF7CDFE00284FF0000045
:10A2800004D0FFF7B7FE4FF44870E5E7FFF7BAFEDA
:10A29000DFE70020FFF7BEFE00284FF0000002D0ED
:10A2A000FFF7A8FECFE7FFF7ADFED4E70020FFF7EA
:10A2B000B1FE00284FF0000002D0FFF79BFE01E046
:10A2C000FFF7A0FE257041F69A1100223868FFF7CB
:10A2D0005DFC064646E00020FFF77AFE257008E0A8
:10A2E000002051E025703DE084F801800120FFF757
:10A2F0006FFE002240F6CD41E8E784F8018001209E
:10A30000FFF766FE00224FF48041DFE77868FFF731
:10A3100081FC0646D5F1110000D02EB10220FFF7D6
:10A3200069FE84F802B01DE0012816D980B2C82168
:10A330004843C117C90341EA5041C0034FF4FA72C0
:10A34000801841F1000152000023FEF7E7FF0146AB
:10A3500000227868FFF71AFC06460220FFF752FE3B
:10A3600084F802803046BDE8F09F00F069FAB9E752
:10A3700000F066FAB4E700F063FA04E000F060FA77
:10A380000020FFF73FFE0120FFF73CFEAAE7FFF7A2
:10A390005AFEA7E7381C00209CBB01000078022170
:10A3A000FFF76CBE05494FF0FF32082841F8202026
:10A3B00002D3084480F8482070470000D41D0020D4
:10A3C000F0B54FF0FF3512B10023082601E0082355
:10A3D0000C260C4C05E000BF54F823707F1C04D001
:10A3E0005B1CB342F8D32846F0BD26185DB286F850
:10A3F000305044F82310002AF5D1E11881F84800C4
:10A40000F1E70000D41D00200249084490F9300013
:10A4100070470000D41D002030B58FB000240546E1
:10A4200007949DF81E001C2120F00600801C8DF86A
:10A430001E009DF81C0020F00F00401C20F0F000D2
:10A4400010308DF81C009DF81D0020F00F00401CFE
:10A4500020F0F00010308DF81D006846FEF7B7FFC1
:10A460009DF80000039440F012008DF8000007A84A
:10A47000CDE904408DF83A5041F22450ADF838004F
:10A480000D949DF83400019420F00F00401C20F042
:10A49000F00010308DF834009DF83500069420F05F
:10A4A000FF008DF835009DF83600142120F00600DD
:10A4B000801C20F019008DF8360008A8FEF787FFF1
:10A4C0000EA808900DA809901420ADF82800ADF84A
:10A4D0002C000848084B0C90A3F10800ADF82A4066
:10A4E00008AA6946C088AADF002801D0FFF706FB4A
:10A4F0000FB030BD081D0020201C002000B585B025
:10A5000017491420ADF810008888A0F57F42FF3A63
:10A5100023D00978002920D00021114B01220833D3
:10A5200000910191ADF810201B88ADF8041004A92A
:10A5300002910C49ADF8003003918DF80220694674
:10A54000AEDF002809D0082807D0132805D043F231
:10A550000141884201D0FFF7D1FA05B000BD0000EB
:10A56000181C0020081D002070B5084C050009D0FB
:10A5700010342168002907D00868206049682846FF
:10A580008847F6E70834F4E770BD0000C01D0020DE
:10A59000054A012120B1012805D19170FFF7E4BFE0
:10A5A00051700020FAE77047C01D00202DE9F05FD0
:10A5B00026484168F1B3DFF898B00E688146DBF8B1
:10A5C000004087688078E11B21F07F45ED1CB0B921
:10A5D000DFF880804FF48030C8F84403C8F80403E3
:10A5E0001120FEF7D3FF1120FEF7DBFF4FF0010A29
:10A5F000C8F800A02F2000F09FFE89F802A0B54205
:10A6000000D23546124BE8193C3320F07F401860E9
:10A61000DBF800105A46091B21F07F41001B20F097
:10A620007F40C91C81420FD9106818602F2000F0AC
:10A6300083FE00E004E0BDE8F05F1120FEF7BCBF40
:10A64000BDE8F05F00F0D0BFBDE8F09F701C0020B7
:10A6500004150140001001402DE9F041178806461D
:10A66000B81D14460D46984202D90C20BDE8F08171
:10A670003188072206290AD34FF4486C4FF6FF733E
:10A68000614501D9994202D17088062801D210464D
:10A69000ECE7604501D99842F9D1994203D098423C
:10A6A00001D08142F3D80520E85520881221401CB2
:10A6B00080B2208029542088401C80B2208041191B
:10A6C000308801F0C3F92188084480B22080411904
:10A6D000708801F0BBF92188084420800020C5E77C
:10A6E000FFF70CBF2DE9F0470025DFF88C803CE038
:10A6F0006068002100EBC506012032789146FEF724
:10A700003EFED4E9062300EA020701EA030C57EAF9
:10A710000C0728D082438B434846C4E9062300F047
:10A72000CDFE32788246914601200021FEF727FEB9
:10A73000D4E9042300EA020401EA03074A4650462A
:10A740000021FEF71CFE44404F403C430BD1707883
:10A75000012801D0012100E00021726881EA0A018C
:10A760000AB1484690476D1CEDB298F80000444687
:10A770008542BDD3BDE8F087501C00200E4910B5BE
:10A780000A784C780023A24212D0521CD2B20A702E
:10A79000022A00D10B70084A0B780C3252F82320A1
:10A7A00002608868104420F07F408860012010BD5E
:10A7B0000360002010BD0000701C00202DE9F04156
:10A7C0008046024601200021FEF7D9FD1A4F0546BA
:10A7D0000E467868FFF71EFA00280CD1174CD4E912
:10A7E000062110462A4001EA06031A4305D0A84371
:10A7F000B143C4E90601BDE8F081404600F05EFEC9
:10A8000030B1D4E9040128433143C4E9040105E02F
:10A81000D4E90410A943B043C4E90410D4E9060103
:10A8200028433143C4E90601A1687868BDE8F041D6
:10A830000022FFF7ABB90000DCBB0100501C002078
:10A840000A4810B5807860B1002401E0022C06D0DF
:10A850002046FFF7CFFB641C042CF7D310BD032464
:10A86000F6E7BDE81040FFF7E5BB0000381C00200C
:10A8700003480179C90702D00078FFF7B3BC7047DD
:10A88000381C002017210180418000210171417195
:10A89000704700002DE9F047394E002780463D46BD
:10A8A000DFF8E090D6F804A057E003D00446D0F8D3
:10A8B0001C8035E099F8002002EB4201521CD2B214
:10A8C00089F8002009EBC10199F80230091D9A426C
:10A8D00001D189F8005048680A780446012A12D04C
:10A8E000022A02D0032A3BD108E001F021F800B18E
:10A8F0000127257434E00574C06900E07068002801
:10A90000F9D170602CE0207C50BB88686060C8681A
:10A91000A0600869E0604869A061F07800B16560F6
:10A920006268B168184B501A20F07F40984202D2FA
:10A93000A168084406E0881AA16820F07F4081429F
:10A9400002D9081A206000E0256065600120A5603A
:10A9500020742046E56100F0CDFFB8F10000A4D1DD
:10A9600099F8001099F801008142A3D117B97168D4
:10A97000514502D00120BDE8F0870020FBE7000030
:10A98000701C0020501E0020FFFF7F000EB5FFF757
:10A99000D3F808B1FFF7B2F85C4A01215C48FFF731
:10A9A000B9F808B1FFF7AAF859485A4A0021001D22
:10A9B000FFF7B0F808B1FFF7A1F800210320FFF777
:10A9C000C7FB08B1FFF79AF800F01EFB08B1FFF7CC
:10A9D00095F80020FFF7C2FA4F4E707018B90120A9
:10A9E000FFF7BCFAB07000F0CDFB08B1FFF786F8B6
:10A9F000002569460120009500F04EFB08B1FFF7E5
:10AA00007DF8684600F086FB08B1FFF777F87078AC
:10AA1000B178084301D100F015FB9DF808003FA173
:10AA200020F00F00401C20F0F00010308DF80800DE
:10AA3000112202A87CDF08B1FFF760F80095102012
:10AA4000ADF800000195ADF80200ADF804504FF4E8
:10AA5000C870ADF8060068467ADF08B1FFF74EF817
:10AA60000021334800F017F908B1FFF747F83148E3
:10AA700000902F486946103000F0AFF908B1FFF799
:10AA80003DF82B4C707801271C34002840F6B8386C
:10AA90004FF01801204622D0FEF799FC2770A4F849
:10AAA0000C80656025752020A060677541F22350F9
:10AAB000ADF8000016480DF10201083062DF08B160
:10AAC000FFF71CF8144A6946921D0120A8DF08B15F
:10AAD000FFF714F89DF80200FFF79EFC0AE0FEF76E
:10AAE00076FC04202070A4F80C8065602575A020F9
:10AAF000A0606775FEF762FF0121F07873DF08B18F
:10AB0000FEF7FCFF00F094FAFCE70000E1A601006C
:10AB10007CBB010039AC0100181C00204E6F726430
:10AB200069635F506F7765725F4D676D74000000F9
:10AB3000D41C002081B0010070B5144682880E46F6
:10AB400005462088111D0144921C994201D8FE2A15
:10AB500001D90C2070BD521C32542088FF21401CAA
:10AB600080B2208031542088401C80B2208081191E
:10AB7000288800F06BFF2188084480B22080AA88D2
:10AB800042B1A96841B13044FEF708FC2088A98889
:10AB900008442080002070BD072070BDF8B50F4626
:10ABA000017814460546012901D1687830B1208822
:10ABB000821C9A422DD8012902D006E00720F8BD58
:10ABC00069780144891C994223D8181A801E86B2DC
:10ABD000ADF800602188B81C084469467DDF002874
:10ABE000EDD12878022805D1BDF80010B14201D876
:10ABF00009210AE00821012805D16878B04202D86D
:10AC0000ADF8000001E0ADF80060BDF80000FE28DE
:10AC100001D90C20F8BD2288401CB8542088401C63
:10AC200080B2208039542088401C2080BDF800105C
:10AC3000084420800020F8BD094810B50068FEF7E0
:10AC4000E9FF08B1FEF75AFF06481321808876DF36
:10AC5000002803D0BDE81040FEF750BF10BD000033
:10AC60007CBB0100181C002008B56A46FEF7D2FA2A
:10AC700008BDC20800F007030120895C9840084025
:10AC8000704710B5C20800F00703885C01249C409F
:10AC90002043885410BD10B560B1C160172120F861
:10ACA000021B20F8021B1B2100F8021BFFF7EAFD24
:10ACB000002010BD0E2010BD2DE9FC4786880C46F3
:10ACC000002E4AD1018801270025102908D011291A
:10ACD00020D0DFF8EC903A2920D0552965D13EE00C
:10ACE000C07B04F10608012802D12088A8F80000E2
:10ACF000B8F80010B8F80200814256D93046A5DFF6
:10AD000010B1112803D050E088F805704DE088F8A4
:10AD100004704DE0A01DFFF7B5FD46E022464089D6
:10AD200034F8061F814200D808466080172800D2F8
:10AD300017206080D06870B1607960B1D9E90010E7
:10AD4000CDE90010ADF802606088ADF80400D3686A
:10AD500069461046984765712571BDE8FC87C08833
:10AD600004F10608172800D21720B8F80010814215
:10AD700000D80846A8F8020088F804502846B8F819
:10AD80000010B5DF98F8050078B9E06868B1D9E936
:10AD90000210CDE90010ADF80260B8F80200ADF87D
:10ADA0000400E268204669469047A07A0028D4D083
:10ADB0002846E188A5DF0028CFD1A572E772CCE74D
:10ADC000C8BB010020B10278DE2A03D008207047FA
:10ADD0000E20704741800020704760B159B1027861
:10ADE000DE2A0AD009684160DE2101704FF6FF714A
:10ADF0004180002070470E207047082070477FB5C3
:10AE0000054600294DD0002D4BD008780C46DE2891
:10AE100047D1A8886188884202D1204600F01BFEF5
:10AE20002888012825D002283BD011283AD0512863
:10AE300037D135F8040F6188884232D1A978A81C2F
:10AE400002292ED1017A042903D0062901D005292F
:10AE500027D10021009102228DF8002001914FF4AA
:10AE6000C07202910391ADF80420007A05280FD03A
:10AE700010E0297A2046012913D1A98842889142FD
:10AE80000FD10121017204B0BDE8704000F0E3BDB4
:10AE9000ADF8041028886946B0DF002801D0616849
:10AEA00088477FBDA88861888842FAD14FF6FF7035
:10AEB00060807FBD00F180400068002800D0012044
:10AEC000704708B500F180400021016000680090E3
:10AED00008BD000070B50B4C207808B185250FE047
:10AEE0000020A06060602061E060074800F006FA82
:10AEF000054600F0A1F908B900F0EAF90120207038
:10AF0000284670BDC01D002091A5010038B5002560
:10AF10008DF800506846FEF78DFE074CE068401E35
:10AF2000E060E06810B900F0F9F9A5709DF8000044
:10AF3000FEF7A4FE38BD0000C01D002070B541EA38
:10AF40004201DDE904564FF0A04441EA830141EAA1
:10AF5000052104EB800041EA0641C0F8001770BDEE
:10AF600070B541EA4201DDE904564FF0A04441EAE0
:10AF7000830141EA052104EB800041EA0641C0F863
:10AF8000001770BD4FF0A04202EB8000D0F8002700
:10AF900022F44032C0F80027D0F8002742EA0141ED
:10AFA000C0F80017704701224FF0A043824011B152
:10AFB000C3F808257047C3F80C25704718B5084B2F
:10AFC0006C4601441B68009306E000BF54F8203033
:10AFD000D3F81035401C08C28142F7D818BD0000D4
:10AFE000D8BB0100034908B508440021016000688E
:10AFF000009008BD0060004002494058012800D080
:10B000000020704700600040064910B500204870DD
:10B01000091D0860BFF35F8F0349044800F030F951
:10B02000002010BD841C002004BC0100681F00200B
:10B0300010B500F001F908B141DF10BD20BF40BFDD
:10B0400020BF10BD70B504460C480121FFF70CFE6F
:10B05000BFF35F8F0025002809D10120074E042C83
:10B0600008D0311F4A781AB1BFF35F8F356070BDC9
:10B070000C70487000F092FBF6E70000881C00207E
:10B08000FEF73CBD20B1034909680160002070470C
:10B090000E20704788BC0100FEB502460C460846EB
:10B0A000FFF7F0FF002834D1002500950195012617
:10B0B00006208DF80020ADF8040002958DF802609E
:10B0C00069462020226869DF0095019502958DF878
:10B0D000016069464020226869DF0095019502956C
:10B0E0008DF8006069460120226869DF4FF4B06086
:10B0F0000090019502956946A120226869DF0095BC
:10B10000019502958DF800506946A020226869DFFC
:10B110000020FEBD60DF002802D1024A012111702B
:10B12000704700008F1C002030B5144891B00078A3
:10B13000002820D05FF03405ADF8405010A903A8D6
:10B1400061DF30B1052816D011B0BDE83040FEF700
:10B15000D5BC03AC0A49684600F092F807E000BF8E
:10B16000D0E9002120469047684600F0A0F80298F8
:10B170000028E1D0F4E711B030BD00008F1C0020A2
:10B180008CBC01007CB5204C207808B108207CBD27
:10B190000120A070002000F08FFA112819D00020A3
:10B1A00000F0A2FA19480026006801908DF80060AE
:10B1B0006846FEF73FFD164901A810DF05000AD0DA
:10B1C000002020709DF80000FEF758FD2DB12846A4
:10B1D0007CBD00207CBD0120F3E7A67066700721CE
:10B1E000162000F01FFA08B1FEF788FC0721152091
:10B1F00000F018FA08B1FEF781FC00F013FB012003
:10B2000000F072FAE5E700008C1C002020BC010071
:10B21000CD9A01000EB50749684600F031F805E007
:10B22000D0E900108847684600F041F802980028ED
:10B23000F6D10EBD3CBC010001480078704700000B
:10B240008C1C00201FB568464BDF30B1052814D098
:10B2500004B0BDE81040FEF751BC084901A800F059
:10B260000FF806E0D0E900210098904701A800F00F
:10B270001EF803980028E6D0F4E71FBDA8BC010023
:10B28000016009684160AFF3008010B5D0E900218A
:10B290005368994201D1002104E0D1E90034A3426E
:10B2A00002D01946816010BD08314160F0E7816825
:10B2B00000290BD0026892680A44826041684B689A
:10B2C0009A4203D108314160FFF7DFBF70470000A9
:10B2D00008480068012110F0010F08D14FF0E0206C
:10B2E000E02280F80024C0F88012C0F80011024863
:10B2F0000160704700E100E0180500400649024681
:10B3000000200B790BB1852070470A6001220A7179
:10B3100000224A7170470000481C002004490120A7
:10B32000086004480168C1F300410029FAD1704760
:10B330000C00004018040040002802D001498001A0
:10B3400008477047E5BB01002DE9F04188460546F6
:10B3500000F032F9234E002828461AD0FFF754F89F
:10B36000304490F848008009032802D001280ED00C
:10B3700007E04FF0A040D0F81005E84010F0010FB2
:10B3800005D003212846BDE8F041FFF7FBBD0221AF
:10B39000F8E700F01DF9002822D02846FFF734F81E
:10B3A00004464FF4807000EB84000F4F81B207EB2E
:10B3B0008400D0F8102542F00102C0F8102508469C
:10B3C000FFF710FEB8F1000F0AD02846FFF71CF86F
:10B3D00056F82000002803D00120A040C7F804033D
:10B3E000BDE8F081D41D0020006000402DE9FC4143
:10B3F000DFF8BC80044608EB0400002790F9300019
:10B400001346C0170E46401C01D008274CE0B07808
:10B410001946C0F340022046FEF7D2FF0546401C05
:10B4200041D0B078410719D4C0070AD04FF0A040EE
:10B4300000EB8401D1F8000720F00200C1F80007FA
:10B4400007E000217378204600910A460191FFF73A
:10B4500087FD174920465431FFF713FCB078800769
:10B4600018D51448317800EB8500D0F81025124B20
:10B470001A40C0F810254FF4F8524FF4403302EA56
:10B48000042203EA01410A43D0F810150A43C0F828
:10B49000102509E008EB0500327810F8481F41EA52
:10B4A0008211017000E004273846BDE8FC810000ED
:10B4B000D41D002000600040FFE0FCFF4FF0A041E1
:10B4C000D1F81015C14011F0010000D001207047E3
:10B4D00070B5184D95F8580008B1082070BD0020CF
:10B4E000411E2A18401CC0B282F830102028F8D320
:10B4F00000242046FEF756FF641CE4B20C2CF8D35F
:10B5000000240D49E0206C6581F8000401264020EC
:10B51000891FC1F88002C1F800014FF4BE70FFF727
:10B5200061FD0649F007C1F8040385F8586020461C
:10B5300070BD0000D41D002006E000E00060004067
:10B54000034890F85800002800D001207047000000
:10B55000D41D002010B5164A30F8061F928891427B
:10B5600024D14189022921D10C30FEF7F3FC104986
:10B5700008390870B0B10F4C002240F28F212068CA
:10B58000FEF704FB08B1FEF7B9FA00224FF42031B0
:10B590006068FEF7FBFA08B1FEF7B0FABDE81040AC
:10B5A000FEF7ACBFBDE81040FEF782BB10BD000047
:10B5B000201C00207CBB01000449084490F93000A5
:10B5C000082801DB0120704700207047D41D0020AF
:10B5D0000449084490F93000082801D2012070473E
:10B5E00000207047D41D002070B5012670044FF074
:10B5F000E0210025C1F88001084C4010C4F8480340
:10B60000C4F8080366602F20FFF796FEA660044C7E
:10B610002F20A560FFF790FEA57070BD00100140BF
:10B62000701C002070B50D460446FEF7A9F970B1F4
:10B630002846FEF7B7F968B16807000E002C0CDA4F
:10B6400004F00F0101F1E02181F8140D09E042F24C
:10B65000010070BD42F2020070BD04F1E02484F8E4
:10B660000004002070BD000038B50021012548B15C
:10B6700001280CD0032809D1FFF72AFEBDE8384085
:10B68000FFF744BC4FF0E020C0F8805138BD8DF882
:10B6900000106846FEF7CEFA064C207808B9FFF78E
:10B6A00019FCE068401CE060A5709DF80000FEF702
:10B6B000E5FA38BDC01D00203EB50446094968467C
:10B6C000FFF7DEFD08E000BFD0E9002120469047EB
:10B6D00030B16846FFF7EBFD02980028F4D13EBD7B
:10B6E00011203EBD24BC01003EB504460849684611
:10B6F000FFF7C6FD07E000BFD0E9002120469047D4
:10B700006846FFF7D4FD02980028F5D13EBD000041
:10B7100030BC01002DE9F0410746806A1446884696
:10B72000C8B3002531E000BFB96A05EB450001EB65
:10B730008006B088801CFE2802D90C20BDE8F0816C
:10B740002288401C08F8020020881622401C80B283
:10B75000208008F800202088401C80B2208000EB68
:10B760000801308800F072F92188084480B22080F6
:10B77000B28842B1B16871B14044FDF70FFE208834
:10B78000B188084420806D1CEDB297F82C00A842C7
:10B79000CAD80020D2E7FFE70720CFE770B5164DE3
:10B7A000164C07E0016820788847002822D012480C
:10B7B000FFF77DFDA8680028F4D1207803280CD07D
:10B7C00002280AD0FFF738FD00B133DF0C49012011
:10B7D0000860BFF34F8F20BFFDE7BFF34F8F0948CD
:10B7E0000168094A01F4E06111430160BFF34F8F22
:10B7F00000BFFDE770BD0000681F0020841C002012
:10B80000000500400CED00E00400FA05002805D119
:10B810000349012048700020FEF7A6BE70470000D3
:10B82000C01D002010B51620FEF7AAF880B10F4801
:10B8300090F800044009FEF7B5F860B10C48826842
:10B840004FF480016AB1016841F48001016010BDCC
:10B8500042F2010001E042F20200BDE81040FEF7B2
:10B860004DB94FF0E020C0F8001110BD16E000E027
:10B870005C1F00202DE9F84F1D4C00256846D4E9D7
:10B8800001A6FEF77BFF002738B30023009A61680A
:10B890001CE0D1F800C00846944503D9ACEB020285
:10B8A0000A6015E0A2EB0C0263440760D0F80CC0FC
:10B8B000C1698146BCF1000F08D006EB030828F0EF
:10B8C0007F48C0E9018CC9F81C5005460029E0D129
:10B8D00028466160FEF7DEFF03E02846FEF7DAFF48
:10B8E00010B15046FEF762FEE770BDE8F88F000029
:10B8F000701C00200D4B10B5596831B102680C68FE
:10B90000A24204D8A21A0A60C161586010BD0B4659
:10B9100003E00B46C969121B21B10C689442F8D3AD
:10B92000A41A0C600260C161D86110BD701C0020B7
:10B930002DE9F041144E77683D462C4603E08442E1
:10B9400004D02546E469002CF9D11BE0D4B1A5420E
:10B950000BD1F869706040B90C4901208860002162
:10B96000B160F0702F20FFF7E7FC2168E069E86123
:10B9700010B10268114401607068874202D0012052
:10B98000BDE8F0810020FBE7701C002000100140A2
:10B990007CB5064600240D468DF800406846FEF74B
:10B9A00049F901A800F06AF870B1057009494660CC
:10B9B0009DF8040048709DF80000FEF75FF9142020
:10B9C000FDF7FAFD20467CBD04249DF80000FEF73B
:10B9D00055F9F7E7501E00202DE9F041194D6C682C
:10B9E000002C2CD0184800270068A968B846401AD7
:10B9F00020F07F462068B0420CD82146361A074412
:10BA0000E469087C20B181F8108088694969884719
:10BA1000002CEFD129786878814206D1401CC0B251
:10BA20006870022801D185F80180064869780C30D9
:10BA300040F82170BDE8F0411420FDF7BDBDBDE820
:10BA4000F0810000701C0020041501400870000AFD
:10BA500048700220704730B40446007A00280AD0AB
:10BA60006088002166DF28B1112802D0616830BCEF
:10BA700008470120207230BC704700000A494A780C
:10BA80008B78521CD2B2934200D100220B789342A1
:10BA900001D1002070470270487800EB400001EBB4
:10BAA000C000001D70470000501E00202DE9FC4121
:10BAB0001646DDE90854CDE900541F4680460222AF
:10BAC00000F00CF8002807D1CDE900543B461022C5
:10BAD0003146404600F002F8BDE8FC812DE9FC5FEC
:10BAE0000026DDE90C4B994692468E468046278813
:10BAF000354630E0D8F80400002200EB85006946A6
:10BB00000068019001A864DF002830D19DF8000092
:10BB100050451FD10EB1002100E0022122880844C7
:10BB20001118594522D846B9521C90B2208009F804
:10BB300000E02088401C20800126218801A801EB1C
:10BB40000902694664DF002811D120889DF80010A1
:10BB5000084420806D1CB8F80000A842CADC56B129
:10BB60002088C01B401E80B2FF2802D90C20BDE8EF
:10BB7000FC9F09F807000020F9E70000941C002052
:10BB8000B41C002023D1BCEA5F782315DEEF12122B
:10BB900000000000111213140D0E0F10541D002090
:10BBA000741D0020A01D00200D0003007DA00100D9
:10BBB0000E0003007DA001000F0003007DA0010026
:10BBC000100003007DA00100770A000000000000C3
:10BBD000770A000000000000000000500300000091
:10BBE000301E00200738FDD870470000000000001C
:10BBF0000000000000000000000000000000000045
:10BC000000000000ECBB010004BC010004000000C7
:10BC10000000000000000000000000000000000024
:10BC20000100000710BC010020BC0100080000005A
:10BC300048BC010058BC01000800000058BC0100CD
:10BC400068BC01000800000004BD01000CBD01003B
:10BC50000000000000000000F4BC010004BD010071
:10BC600000000000000000000000000000000000D4
:10BC7000D4BC0100DCBC0100DCBC0100E4BC010060
:10BC8000E4BC0100ECBC0100181C002068BC0100F1
:10BC900088BC010008000000ECBC0100F4BC0100FD
:10BCA000000000000000000098BC0100A8BC0100DA
:10BCB000080000000CBD0100181C00207C000000E2
:10BCC0006099010088BD0100941C0020E40A000076
:10BCD00070990100B9AC0100D41C0020FFAD010037
:10BCE000E41C0020BD9E0100000000000DB8010012
:10BCF0000000000029B101000000000045B2010071
:10BD00000000000069B6010000000000000000FF14
:10BD1000FFFF00000000000000000000341D0020B4
:10BD20001F000000000000000000000000000000F4
:10BD30000000000000000000000000000000000003
:10BD400000000000000000000000000000000000F3
:10BD500000000000000000000000000000000000E3
:10BD600000000000000000000000000000000000D3
:10BD700000000000000000000000000000000000C3
:08BD8000000000000090D00358
:040000050001920163
:00000001FF
